
 Start  Stop   Length Name               Class

 00000H 05EB9H 05EBAH CODE               

  Address         Publics by Name

 0000:4D60       AADDR_MSG
 0000:47A6       ALREADY_MSG
 0000:0A50       AS_SEND_PKT
 0000:52F0       BUSTYPE_PARA_TABLE
 0000:52D5       BUSTYPE_TABLE
 0000:524F       BYTEOUT
 0000:52F6       B_10BASET
 0000:52FE       B_AUI
 0000:0925       B_BUSTYPE
 0000:0924       B_CPUFLAG
 0000:5302       B_FDUP_OFF
 0000:52E2       B_ISA_BUS
 0000:52AB       B_KBUSTYPE
 0000:52A1       B_KDMAROTATE
 0000:52CC       B_KDMATIMER
 0000:5293       B_KDMA_NO
 0000:52C7       B_KFDUP
 0000:528B       B_KINT_NO
 0000:5297       B_KIOADDR_NO
 0000:528F       B_KIRQ_NO
 0000:52B3       B_KLED0
 0000:52B8       B_KLED1
 0000:52BD       B_KLED2
 0000:52C2       B_KLED3
 0000:529E       B_KTP_EN
 0000:0926       B_OEM1
 0000:0927       B_OEM2
 0000:0928       B_OEM2_ENABLE
 0000:52E6       B_PCI1_BUS
 0000:52EB       B_PCI2_BUS
 0000:52D5       B_PCI_BUS
 0000:093F       B_PCI_METHOD
 0000:52DE       B_PNP_BUS
 0000:52D9       B_VESA_BUS
 0000:5270       CHROUT
 0000:4C39       COPYLEFT_MSG
 0000:4C0C       COPYRIGHT_MSG
 0000:06E9       COUNT_IN_ERR
 0000:06F6       COUNT_OUT_ERR
 0000:4D76       CRLF_MSG
 0000:51FE       DECOUT
 0000:5600       DEVICES_INIT
 0000:525E       DIGOUT
 0000:5D36       DISPLAY_ERROR_MESSAGE
 0000:09A9       DMA_NO
 0000:09AD       DRIVER_CLASS
 0000:09B8       DRIVER_FUNCTION
 0000:09B1       DRIVER_NAME
 0000:09B0       DRIVER_TYPE
 0000:0A51       DROP_PKT
 0000:5241       DWORDOUT
 0000:0943       DW_PCI_BDFNUM
 0000:4D48       EADDR_MSG
 0000:0920       EISA_SIGN_STR
 0000:5323       ERROR
 0000:4C00       ERROR_HEADER
 0000:4E15       ETOPEN
 0000:528A       ETOPEN_DIAGN
 0000:010A       FLAGBYTE
 0000:5306       FULLDUPLEX_PARA_TABLE
 0000:52F6       FULLDUPLEX_TABLE
 0000:0B20       GET_ADDRESS
 0000:55A4       GET_DIGIT
 0000:553C       GET_HEX
 0000:5537       GET_NUMBER
 0000:4876       INIT_ERR0_MSG
 0000:4A1C       INIT_ERR10_MSG
 0000:4A49       INIT_ERR11_MSG
 0000:4A75       INIT_ERR12_MSG
 0000:4AA1       INIT_ERR13_MSG
 0000:4AC4       INIT_ERR14_MSG
 0000:4AE7       INIT_ERR15_MSG
 0000:4AFC       INIT_ERR16_MSG
 0000:4B11       INIT_ERR17_MSG
 0000:4B26       INIT_ERR18_MSG
 0000:4B3B       INIT_ERR19_MSG
 0000:48A8       INIT_ERR1_MSG
 0000:48DB       INIT_ERR2_MSG
 0000:4901       INIT_ERR3_MSG
 0000:4927       INIT_ERR4_MSG
 0000:494E       INIT_ERR5_MSG
 0000:4974       INIT_ERR6_MSG
 0000:498C       INIT_ERR7_MSG
 0000:49B1       INIT_ERR8_MSG
 0000:49F0       INIT_ERR9_MSG
 0000:47D2       INT_MSG
 0000:47F8       INT_MSG_NUM
 0000:09A1       INT_NO
 0000:09A5       IO_ADDR
 0000:0108       IS_AT
 0000:528B       KEYWORD_STRING_TABLE
 0000:4D12       LOCATION_MSG
 0000:0783       MASKINT
 0000:0238       MULTICAST_ADDRS
 0000:0232       MULTICAST_BROAD
 0000:0230       MULTICAST_COUNT
 0000:4807       NO_RESIDENT_MSG
 0000:02B1       OUR_ISR
 0000:483B       PACKET_INT_MSG
 0000:0104       PACKET_INT_NO
 0000:4D2F       PACKET_INT_NUM
 0000:09B9       PARAMETER_LIST
 0000:4D79       PARSE_ARGS
 0000:0080       PHD_DIOA
 0000:002C       PHD_ENVIRON
 0000:55D9       PRINT_ETHER_ADDR
 0000:51CA       PRINT_NUMBER
 0000:5020       PRINT_PARAMETERS
 0000:09C7       RCV_MODES
 0000:0C32       RECV
 0000:088D       RECV_COPY
 0000:0DAA       RECV_EXITING
 0000:07D5       RECV_FIND
 0000:0C31       RESET_INTERFACE
 0000:031A       RE_ENABLE_INTERRUPTS
 0000:08E2       SEND_DEQUEUE
 0000:0285       SEND_HEAD
 0000:0A53       SEND_PKT
 0000:08A7       SEND_QUEUE
 0000:0289       SEND_TAIL
 0000:0B3B       SET_ADDRESS
 0000:0BEB       SET_MULTICAST_LIST
 0000:06C0       SET_RECV_ISR
 0000:0E16       SHARE_ISR
 0000:55CA       SKIP_BLANKS
 0000:535C       START_1
 0000:0109       SYS_FEATURES
 0000:0BEF       TERMINATE
 0000:02AD       THEIR_ISR
 0000:07A6       UNMASKINT
 0000:4B50       USAGE_MSG
 0000:5248       WORDOUT
 0000:0A52       XMIT

  Address         Publics by Value

 0000:002C       PHD_ENVIRON
 0000:0080       PHD_DIOA
 0000:0104       PACKET_INT_NO
 0000:0108       IS_AT
 0000:0109       SYS_FEATURES
 0000:010A       FLAGBYTE
 0000:0230       MULTICAST_COUNT
 0000:0232       MULTICAST_BROAD
 0000:0238       MULTICAST_ADDRS
 0000:0285       SEND_HEAD
 0000:0289       SEND_TAIL
 0000:02AD       THEIR_ISR
 0000:02B1       OUR_ISR
 0000:031A       RE_ENABLE_INTERRUPTS
 0000:06C0       SET_RECV_ISR
 0000:06E9       COUNT_IN_ERR
 0000:06F6       COUNT_OUT_ERR
 0000:0783       MASKINT
 0000:07A6       UNMASKINT
 0000:07D5       RECV_FIND
 0000:088D       RECV_COPY
 0000:08A7       SEND_QUEUE
 0000:08E2       SEND_DEQUEUE
 0000:0920       EISA_SIGN_STR
 0000:0924       B_CPUFLAG
 0000:0925       B_BUSTYPE
 0000:0926       B_OEM1
 0000:0927       B_OEM2
 0000:0928       B_OEM2_ENABLE
 0000:093F       B_PCI_METHOD
 0000:0943       DW_PCI_BDFNUM
 0000:09A1       INT_NO
 0000:09A5       IO_ADDR
 0000:09A9       DMA_NO
 0000:09AD       DRIVER_CLASS
 0000:09B0       DRIVER_TYPE
 0000:09B1       DRIVER_NAME
 0000:09B8       DRIVER_FUNCTION
 0000:09B9       PARAMETER_LIST
 0000:09C7       RCV_MODES
 0000:0A50       AS_SEND_PKT
 0000:0A51       DROP_PKT
 0000:0A52       XMIT
 0000:0A53       SEND_PKT
 0000:0B20       GET_ADDRESS
 0000:0B3B       SET_ADDRESS
 0000:0BEB       SET_MULTICAST_LIST
 0000:0BEF       TERMINATE
 0000:0C31       RESET_INTERFACE
 0000:0C32       RECV
 0000:0DAA       RECV_EXITING
 0000:0E16       SHARE_ISR
 0000:47A6       ALREADY_MSG
 0000:47D2       INT_MSG
 0000:47F8       INT_MSG_NUM
 0000:4807       NO_RESIDENT_MSG
 0000:483B       PACKET_INT_MSG
 0000:4876       INIT_ERR0_MSG
 0000:48A8       INIT_ERR1_MSG
 0000:48DB       INIT_ERR2_MSG
 0000:4901       INIT_ERR3_MSG
 0000:4927       INIT_ERR4_MSG
 0000:494E       INIT_ERR5_MSG
 0000:4974       INIT_ERR6_MSG
 0000:498C       INIT_ERR7_MSG
 0000:49B1       INIT_ERR8_MSG
 0000:49F0       INIT_ERR9_MSG
 0000:4A1C       INIT_ERR10_MSG
 0000:4A49       INIT_ERR11_MSG
 0000:4A75       INIT_ERR12_MSG
 0000:4AA1       INIT_ERR13_MSG
 0000:4AC4       INIT_ERR14_MSG
 0000:4AE7       INIT_ERR15_MSG
 0000:4AFC       INIT_ERR16_MSG
 0000:4B11       INIT_ERR17_MSG
 0000:4B26       INIT_ERR18_MSG
 0000:4B3B       INIT_ERR19_MSG
 0000:4B50       USAGE_MSG
 0000:4C00       ERROR_HEADER
 0000:4C0C       COPYRIGHT_MSG
 0000:4C39       COPYLEFT_MSG
 0000:4D12       LOCATION_MSG
 0000:4D2F       PACKET_INT_NUM
 0000:4D48       EADDR_MSG
 0000:4D60       AADDR_MSG
 0000:4D76       CRLF_MSG
 0000:4D79       PARSE_ARGS
 0000:4E15       ETOPEN
 0000:5020       PRINT_PARAMETERS
 0000:51CA       PRINT_NUMBER
 0000:51FE       DECOUT
 0000:5241       DWORDOUT
 0000:5248       WORDOUT
 0000:524F       BYTEOUT
 0000:525E       DIGOUT
 0000:5270       CHROUT
 0000:528A       ETOPEN_DIAGN
 0000:528B       KEYWORD_STRING_TABLE
 0000:528B       B_KINT_NO
 0000:528F       B_KIRQ_NO
 0000:5293       B_KDMA_NO
 0000:5297       B_KIOADDR_NO
 0000:529E       B_KTP_EN
 0000:52A1       B_KDMAROTATE
 0000:52AB       B_KBUSTYPE
 0000:52B3       B_KLED0
 0000:52B8       B_KLED1
 0000:52BD       B_KLED2
 0000:52C2       B_KLED3
 0000:52C7       B_KFDUP
 0000:52CC       B_KDMATIMER
 0000:52D5       BUSTYPE_TABLE
 0000:52D5       B_PCI_BUS
 0000:52D9       B_VESA_BUS
 0000:52DE       B_PNP_BUS
 0000:52E2       B_ISA_BUS
 0000:52E6       B_PCI1_BUS
 0000:52EB       B_PCI2_BUS
 0000:52F0       BUSTYPE_PARA_TABLE
 0000:52F6       FULLDUPLEX_TABLE
 0000:52F6       B_10BASET
 0000:52FE       B_AUI
 0000:5302       B_FDUP_OFF
 0000:5306       FULLDUPLEX_PARA_TABLE
 0000:5323       ERROR
 0000:535C       START_1
 0000:5537       GET_NUMBER
 0000:553C       GET_HEX
 0000:55A4       GET_DIGIT
 0000:55CA       SKIP_BLANKS
 0000:55D9       PRINT_ETHER_ADDR
 0000:5600       DEVICES_INIT
 0000:5D36       DISPLAY_ERROR_MESSAGE

Program entry point at 0000:0100
Warning: No stack

